:100000001FC036C435C434C433C432C431C430C450
:100010002FC42EC42DC42CC42BC42AC429C428C464
:1000200027C426C425C424C423C422C421C420C494
:100030001FC41EC43F003F10803F103F1400087AC9
:1000400011241FBECFEFCDBFDFE3DEBFE4E3F0E05E
:1000500040E017C0B591A59135912591059107FD17
:100060000CC095918591EF01F92FE82F05900D9225
:10007000A217B307D9F7FE0104C01D92A217B30758
:10008000E1F7E034F40731F707D2A8C3F894FFCFC3
:100090004F925F926F927F928F929F92AF92BF9298
:1000A000CF92DF92EF92FF92CF936B017C0123EE10
:1000B00038E34EE85FE3DAD34B015C0120E030E047
:1000C00040E85FE3C0D388230CF464C024E535E541
:1000D00045E55FE3C701B601C9D32B013C0120E030
:1000E0003FEF4FE757E4B3D318160CF03EC020E0C3
:1000F00030E04AE754E4C701B601B6D34B015C01D6
:1001000024E535E540E554E4B1D36B017C0120E002
:1001100030E040E85FE397D388230CF120E03FEF25
:100120004FE757E4C701B60192D31816A4F420E0B4
:1001300030E040E251E4C501B40198D3DFD161154C
:10014000710549F123E530E0C9010197F1F76150EC
:100150007109D1F720C0C701B601D0D102C061E05A
:1001600070E0CB010197F1F716C020E030E04FE7D7
:1001700053E4C501B4016BD318163CF4C301B201BA
:10018000BDD1CB010197F1F709C0C501B401B6D1CA
:10019000C62F01C0C1E06C2F6A95F1F7CF91FF9097
:1001A000EF90DF90CF90BF90AF909F908F907F9017
:0801B0006F905F904F900895DD
:1001B8000BC002D340F0F9D230F021F45F3F19F0C0
:1001C80016C3511101C349C30BD298F39923C9F33C
:1001D8005523B1F3951B550BBB27AA276217730745
:1001E800840738F09F5F5F4F220F331F441FAA1FF9
:1001F800A9F333D00E2E3AF0E0E830D091505040B9
:10020800E695001CCAF729D0FE2F27D0660F771F66
:10021800881FBB1F261737074807AB07B0E809F048
:10022800BB0B802DBF01FF2793585F4F2AF09E3FDD
:10023800510568F0DCC2C8C25F3FECF3983EDCF3BE
:10024800869577956795B795F7959F5FC9F7880F56
:10025800911D9695879597F90895E1E0660F771FA8
:10026800881FBB1F621773078407BA0720F0621B39
:0E027800730B840BBA0BEE1F88F7E095089508
:100286000AC094D228F099D218F0952309F0B0C28A
:10029600E5C211249AC2A5D1A0F3959FD1F3950F7B
:1002A60050E0551F629FF001729FBB27F00DB11DF4
:1002B600639FAA27F00DB11DAA1F649F6627B00D84
:1002C600A11D661F829F2227B00DA11D621F739F6D
:1002D600B00DA11D621F839FA00D611D221F749F7B
:1002E6003327A00D611D231F849F600D211D822FC2
:1002F600762F6A2F11249F5750408AF0E1F0882309
:100306004AF0EE0FFF1FBB1F661F771F881F915015
:100316005040A9F79E3F510570F06AC256C25F3F32
:10032600ECF3983EDCF3869577956795B795F79548
:10033600E7959F5FC1F7FE2B880F911D96958795D0
:0403460097F9089586
:10034A00E89409C097FB3EF4909580957095619565
:10035A007F4F8F4F9F4F9923A9F0F92F96E9BB271B
:10036A009395F695879577956795B795F111F8CF97
:10037A00FAF4BB0F11F460FF1BC06F5F7F4F8F4F02
:10038A009F4F16C0882311F096E911C0772321F0F8
:10039A009EE8872F762F05C0662371F096E8862F90
:1003AA0070E060E02AF09A95660F771F881FDAF7E7
:0A03BA00880F9695879597F908952E
:1003C4001F93CF93DF93C82F162F8CD1D0E0FE015B
:1003D400E85FF04C2081222329F0612F84E094E02F
:1003E400C0D11FC09C0121503109273E334048F041
:1003F400612F84E094E0B5D1C85FD04C81E088835C
:1004040010C08438934048F4612F80E094E0C3D155
:10041400612F84E094E0BFD104C0612F84E094E0B4
:0A042400A0D1DF91CF911F91089540
:10042E001F93CF93DF93C82F162F57D1D0E0FE0125
:10043E00E050F14C2081222329F0612F84E294E0D8
:10044E008BD11FC09C0121503109273E334048F00B
:10045E00612F84E294E080D1C050D14C81E088833A
:10046E0010C08438934048F4612F80E294E08ED11E
:10047E00612F84E294E08AD104C0612F84E294E07B
:0A048E006BD1DF91CF911F9108950B
:1004980073D1C7D1C7D0C2E0D8E80CE018E80F2E56
:1004A800FAEDEF2EFAE1FF2EF02DC5D1C701019725
:1004B800F1F7BCD18991999137D1C017D107A9F724
:1004C80088EA91E623E530E0F9013197F1F70197E1
:1004D800D9F7C1D0B0D1CAEDDAE1CE010197F1F771
:1004E80062E084E06BDF63E085E09DDF62E086E048
:0404F8009ADFF3CFC5
:1004FC007DD088F09F5790F0B92F9927B751A0F075
:10050C00D1F0660F771F881F991F1AF0BA95C9F79B
:10051C0012C0B13081F055D1B1E0089552C1672FAE
:10052C00782F8827B85F39F0B93FCCF3869577954B
:10053C006795B395D9F73EF4909580957095619534
:08054C007F4F8F4F9F4F089570
:100554000F931F93CF93DF9346D1E091123FF09115
:10056400133F87E009958C0154D13DD1E091123FAE
:10057400F091133F87E00995EC014BD1C11582E05E
:10058400D80730F081E0C017D10718F480E001C02B
:0C05940080E0DF91CF911F910F9108953E
:1005A000990F0008550FAA0BE0E8FEEF1616170684
:1005B000E807F907C0F012161306E407F50798F0EC
:1005C000621B730B840B950B39F40A2661F0232B05
:1005D000242B252B21F408950A2609F4A140A69581
:0805E0008FEF811D811D0895BC
:1005E80057FD9058440F551F59F05F3F71F04795DC
:1005F800880F97FB991F61F09F3F79F087950895C1
:10060800121613061406551FF2CF4695F1DF08C0DF
:10061800161617061806991FF1CF869571056105FC
:040628000894089595
:10062C0060E080E096E014D165E081E096E010D1C6
:10063C0064E082E096E0ABD062E082E096E0A7D086
:10064C0060E483E096E0E6D064E083E096E09FD03F
:02065C000895FF
:10065E0062E080E094E09AD063E080E294E096D08D
:10066E0062E080E294E092D062E084E094E08ED08A
:10067E0063E084E294E08AD062E084E294E086D083
:02068E000895CD
:1006900061E088E096E0E2D0E0E0F6E0838580FF6C
:1006A000FDCFE0E0F6E081E083878089918996952F
:1006B0008795929582958F7089279F7089270895D5
:1006C000CF93883078F4C82F682F80E094E04BD027
:1006D0006C2F84E094E047D08C2F90E064E0805F42
:0806E0009B4F5BD0CF91089500
:1006E800CF93DF93C82FE8DF8DD08C2F2BD0E091EC
:1006F800123FF091133F8C2F0995EC0188D0CE0161
:06070800DF91CF9108957E
:10070E00092E0394000C11F4882352F0BB0F40F411
:10071E00BF2B11F460FF04C06F5F7F4F8F4F9F4F51
:02072E0008952C
:10073000BC0180E090E009DEE091103FF091113FB4
:0C074000099561E084E094E00ED008957B
:10074C00CF93883040F4C82F86E096E07ED06C2F93
:0A075C0086E096E07DD0CF9108956D
:1007660021E030E002C0220F331F6A95E2F72095A0
:0A077600FC01308123232083089545
:1007800062E084E094E0EFDF63E084E294E0EBDF9A
:0A07900062E084E294E0E7DF0895E0
:10079A0021E030E002C0220F331F6A95E2F7FC0124
:0807AA003081232B2083089508
:0E07B20000240A941616170618060906089564
:0E07C00000240A941216130614060506089566
:0E07CE00E894BB2766277727CB0197F908959B
:0E07DC00EC014AD048D0CE0148D0CE0147D023
:0C07EA0087E069DF87E0ADDF0CD00895E8
:0C07F60097F99F6780E870E060E00895CC
:0A080200FA00F401EE02E803E2043C
:0A080C0060E080E096E0C3DF08958D
:0A08160060E080E096E0A4DF0895A2
:0A082000FC012081622B6083089523
:0A082A0061E080E094E0B4DF08957F
:0A08340061E084E094E0AFDF089576
:08083E008ADE8823E9F3089526
:08084600ACDE08F481E0089526
:08084E00A8DE08F48FEF089505
:06085600FC011082089570
:06085C00FC016083089519
:060862009FEF80EC0895F9
:04086800A7DC51CFE9
:04086C000CDD4FCF81
:02087000C7CBF4
:020872000895E7
:020874000895E5
:020876000895E3
:0208780009DC99
:02087A00480034
:02087C0048032F
:00000001FF
